:0A227C00000102020303040405053B
:100C9200E4F513F512F511F510C20EC20BC20DC226
:100CA2000C122183120AA07E1A7F008E5C8F5D7562
:100CB200641A756512755A1A755B1C75621A75632A
:100CC2005175661A75677FEE54E07003020DD9758F
:100CD20014007515808E168F17C374A99FFF741A9E
:100CE2009ECF2402CF3400FEE48F0F8E0EF50DF559
:100CF2000CF50BF50AF509F508AF0FAE0EAD0DAC0C
:100D02000CAB0BAA0AA909A808C3120F325026E598
:100D120015250BF582E514350AF58374CDF0E50B44
:100D22002401F50BE4350AF50AE43509F509E43541
:100D320008F50880C4E4F50BF50AF509F508AF0FCC
:100D4200AE0EAD0DAC0CAB0BAA0AA909A808C312D2
:100D52000F325031AE0AAF0BE5172FF582E5163E82
:100D6200F583E0FDE5152FF582E5143EF583EDF000
:100D7200EF2401F50BE43EF50AE43509F509E43503
:100D820008F50880B985145C85155D74002480FF20
:100D9200741A34FFFEC3E5659FF565E5649EF5644C
:100DA200C3E55F9FF55FE55E9EF55EC3E5619FF576
:100DB20061E5609EF560C3E55B9FF55BE55A9EF5D4
:100DC2005AC3E5639FF563E5629EF562C3E5679FDB
:100DD200F567E5669EF566D2E843D82090E668E0BE
:100DE2004409F090E65CE0443DF0D2AFD288D28A6A
:100DF200C2A8C2AA43E808D2FB90E680E020E1053F
:100E0200D20F121F4C90E680E054F7F0538EF8C2D6
:100E12000E300C05120676C20C300E291218FD5047
:100E220024C20E1220CF200B1690E682E030E70497
:100E3200E020E1EF90E682E030E604E020E0E41218
:0A0E42001FA81222BA12131480C771
:1006760090E6B9E070030207271470030207A4246A
:10068600FE700302082724FB70030207211470037F
:1006960002071B1460731460762405600302088643
:1006A6001222BC400302089290E6BBE024FE6022C0
:1006B60014603324FD601114602224067048E55C42
:1006C60090E6B3F0E55D8037E56490E6B3F0E56566
:1006D600802DE55E90E6B3F0E55F8023E56090E669
:1006E600B3F0E561801990E6BAE0FF121FD4AA06BE
:1006F600A9077B01EA494B600DEE90E6B3F0EF9057
:10070600E6B4F002089202088B12221D0208921229
:1007160022A1020892121D8202089212220B0208DE
:10072600921222BE400302089290E6B8E0247F604F
:100736001514601924027063A20BE43325E0FFA2AE
:100746000DE4334F8041E490E740F0803F90E6BCF3
:10075600E0547EFF7E00E0D394807C0040047D015F
:1007660080027D00EC4EFEED4F247CF58274223E25
:10077600F583E493FF3395E0FEEF24A1FFEE34E624
:100786008F82F583E0540190E740F0E4A3F090E611
:100796008AF090E68B7402F002089202088B12220D
:1007A600C0400302089290E6B8E024FE60162402D8
:1007B600600302089290E6BAE0B40105C20B020893
:1007C6009202088B90E6BAE0705590E6BCE0547E43
:1007D600FF7E00E0D394807C0040047D0180027D92
:1007E60000EC4EFEED4F247CF58274223EF583E448
:1007F60093FF3395E0FEEF24A1FFEE34E68F82F5FA
:1008060083E054FEF090E6BCE05480131313541FAB
:10081600FFE0540F2F90E683F0E04420F0806D80D7
:10082600641222C2506690E6B8E024FE60192402E3
:10083600705A90E6BAE0B40104D20B804F90E6BA43
:10084600E064026047803E90E6BCE0547EFF7E0096
:10085600E0D394807C0040047D0180027D00EC4E54
:10086600FEED4F247CF58274223EF583E493FF333C
:1008760095E0FEEF24A1FFEE34E68F82F583800833
:10088600120080500790E6A0E04401F090E6A0E058
:030896004480F0AB
:01089900223C
:030033000222B6F0
:0422B60053D8EF32D8
:10218300758CE0758AC0E58954F04401F589758E34
:0821930003D28CD2A9D2AF22C5
:03005B0002089AFE
:10089A00C0E0C083C082C0D075D000C004C006C00A
:0108AA000746
:1008AB00AF91530780EF64806003020A9153917FED
:1008BB00300903020A8FE54E64047070D3E53E9451
:1008CB00C8E53D94005003020A8F0537E53725E054
:1008DB002472F582E43424F583E53DF0A3E53EF084
:1008EB00E53725E02470F582E43424F583E0FEA39C
:1008FB00E0FFD394C8EE9400402FEF25E0FFEE33DA
:10090B00FEEF2444FFEE34FDFEE53725E02472F5BF
:10091B0082E43424F583E0FCA3E0D39FEC9E4009F2
:10092B00752D01754E00753700020A89E54E64017D
:10093B0060030209EFD3E53E94C8E53D94005003F4
:10094B00020A8F0537E53725E02472F582E434245B
:10095B00F583E53DF0A3E53EF0E53725E02470F5A2
:10096B0082E43424F583E0FEA3E0FFD394C8EE9435
:10097B0000406EEF25E0FFEE33FEEF2444FFEE3434
:10098B00FDFEE53725E02472F582E43424F583E09F
:10099B00FCA3E0D39FEC9E4048054FE54F640270EB
:1009AB003DE53714F534752D01E53725E0246EF55B
:1009BB0082E43424F583E0FEA3E024C8F539E43E59
:1009CB00F538E53725E02470F582E43424F583E02F
:1009DB00FEA3E024C8F546E43EF545754E00753799
:1009EB0000020A89E54E64027061C3E53E94C8E5D6
:1009FB003D94004048D3E53E94C8E53D940040103B
:100A0B00D3E53E9546E53D95455005752D00802770
:100A1B00D3E53E9546E53D9545400FD3E53E9539EB
:100A2B00E53D95385004052D800DD3E53E9539E510
:100A3B003D95384008052D753D00753E00E52D654B
:100A4B002E7041F54EF53DF53E8039E54EB405343B
:100A5B00D3E53E9401E53D94004029E53725E0249C
:100A6B0072F582E43424F583E53DF0A3E53EF00511
:100A7B0037052DE52DB40F06754E00752D00753D10
:060A8B0000753E00C209E7
:0F0A9100D007D006D004D0D0D082D083D0E032AE
:101A000012010002000000401816019000000102BF
:101A100000010A0600020000004001000902350032
:101A200001010080FA0904000005FF00000007051D
:101A30000102400000070582020002000705810242
:101A400040000007058602000200070508020002A8
:101A50000009022E0001010080FA0904000004FFC1
:101A60000000000705010240000007058202400057
:101A70000007050202000200070581024000000481
:101A800003090410035100480059002D004300438E
:101A90000044001603490043002D00300039003097
:0B1AA00000300030004100200000007A
:10041900608025AC05070202020402070000000201
:10042900000002000A2B0B13111515110000000022
:100439000000003F040A0202020301070000001045
:10044900020002000A2B0B130B1515110000000006
:100459000000003F050F0203030402070000000229
:10046900000002000A2B0B131115111100000000E6
:100479000000003F050F010303040107000000000D
:10048900020002000A2B0B130B15151100000000C6
:100499000000003F60242633000000000000000037
:1004A9000000000000000000000000000000000043
:1004B90000000000000000000000000047262C801A
:0604C900000011EA4E00E4
:1017690090E60174EAF090E6F574FFF090262CE01B
:1017790090E6F3F090262DE090E6C3F090262EE057
:1017890090E6C1F090262FE090E6C2F0902631E075
:1017990090E6C0F0902632E090E6F4F075AF077459
:1017A90025F59A74ACF59B759DE4E4F59EFF90E6EA
:1017B9007BE090E67CF00FBF80F490E67174FFF057
:1017C900F5B490E672E04480F043B680000000E48E
:1017D90090E6C4F000000090E6C5F0902633E09052
:1017E900E6C6F0902634E090E6C7F0902635E09002
:1017F900E6C8F0902636E090E6C9F0902637E090EA
:10180900E6CAF0902638E090E6CBF0902639E090D1
:0B181900E6CCF090263AE090E6CDF01F
:0118240022A1
:030043000219009F
:030053000219008F
:1019000002219B000221E1000221CB000221B30051
:10191000021E18000219B8000218FF000222C400BB
:101920000222C5000222C600021EEA000214FB00C9
:101930000222C7000222C8000222C9000222CA00F5
:101940000222CB000222C4000222CC000222CD00DF
:101950000222CE000222CF000222D0000222D100B9
:101960000222D2000222C4000222C4000222C400C9
:101970000222D3000222D4000222D5000222D60085
:101980000222D7000222D8000222D9000222DA0065
:101990000222DB000222DC000222DD000222DE0045
:1019A0000222DF000222E0000222E1000222E20025
:0819B0000222E3000222E40020
:101FA80090E682E030E004E020E60B90E682E03044
:101FB800E119E030E71590E680E04401F07F147EF7
:0C1FC800001218B790E680E054FEF022F2
:1020CF0090E682E044C0F090E681F0438701000083
:0420DF0000000022DB
:101F4C00300F0990E680E0440AF0800790E680E0CC
:101F5C004408F07FDC7E051218B790E65D74FFF044
:0F1F6C0090E65FF05391EF90E680E054F7F0229B
:021FD400A9075B
:101FD600AE66AF678F828E83A3E064037017AD0190
:101FE60019ED7001228F828E83E07C002FFDEC3E7E
:091FF600FEAF0580DF7E007F00D4
:011FFF0022BF
:1018B7008E1C8F1D90E600E054187012E51D240160
:1018C700FFE4351CC313F51CEF13F51D801590E6D7
:1018D70000E05418FFBF100BE51D25E0F51DE51CC2
:1018E70033F51CE51D151DAE1C7002151C4E600559
:0618F7001220E380EE2246
:1020E3007400F58690FDA57C05A3E582458370F910
:0120F30022CA
:1004CF0060A5250518244242424242424224183E6A
:1004DF0008080808080808080E087E4204081020BB
:1004EF00204242423C1C2242404020182042423CC3
:1004FF007820207E222224242830201C22424040B3
:10050F00261A0202027E1824424242261A020224AE
:10051F0038080808080808101022227E3C42424280
:10052F002418244242423C1C244040586442424218
:10053F0024180000000000FE00000000001C3253D1
:10054F004D4141414141221CE7424242427E4242DB
:10055F004242E71C08080808081414222277E742D1
:10056F0042223C241414180808C1824225AA000014
:10057F004224F200004224F40000412410004124E0
:10058F0011004124FB0002321040C107C104014B8E
:10059F0000012500442501000000004424F700005D
:1005AF000000013C004124F600608024720000002E
:1005BF00000000000000000000000000000000002C
:1005CF00000000000000000000000000000000001C
:1005DF00000000000000000000000000000000000C
:1005EF0000000000000000000000000000000000FC
:1005FF0000000000000000000000000000000000EC
:10060F0000000000000000000000000000000000DB
:10061F0000000000000000000000000000000000CB
:10062F000000000000000000000000000001370083
:10063F00014E01012EFF012D00023D00000134008B
:10064F00014F000238000002450000014D00025426
:10065F0000000235C350012C19C189013100C101BD
:06066F00014100013F0003
:101F7B008E188F199024527403F0E4A3F07A247B0B
:101F8B00527D027F4112214C9024527401F0A3E543
:0D1F9B0019F07A247B527D027F4102214C17
:0B19F500C2B6C2B48FB1D2B4D2B62289
:0B227100D2B6C2B48FB1D2B4D2B622F4
:04216800AE05AD070C
:10216C00E4FCE4FBAF05122271AF061222710BBB2B
:06217C0060F20CBC40EC17
:01218200223A
:10202B00AE05AD077F151219F5AF061219F57F5FD7
:10203B001219F57F751219F5AF051219F57F3F12BD
:0A204B0019F57F251222710222719F
:041BBF007D027F30F4
:021BC300AE036F
:101BC500EDC454F0F518EE75F008A4F519BF2D0411
:101BD5007A0A8020BF51047A0B8019BF48047A0C19
:101BE5008012BF59047A0D800BBF41047A0E800420
:101BF500EF24D0FAE4FBEA75F00BA42405F582E4A2
:101C05003425F583E5822BF582E43583F583E0F908
:101C1500E4FCE930E70DE51824022BFFE5192CFD5E
:0F1C250012202BE925E0F90CBC08E70BBB0BC71D
:011C3400228D
:1020F400C2B77FC87E00121752D2B77FAE1219F54D
:0F2104007FA01219F57F601219F57FAF0219F550
:101825001220F4E4FDFF1221687B097D027F51122D
:101835001BC37B087D027F48121BC37B077D027F8C
:1018450059121BC37B06121BBF7B057D027F391214
:101855001BC37B04121BBF7B03121BBF7B02121B26
:10186500BF7B017D027F41121BC37B097D017F3157
:10187500121BC37B087D017F38121BC37B077D01CB
:101885007F2D121BC37B067D017F30121BC37B0599
:101895007D017F39121BC37B047D017F2D121BC384
:1018A5007B037D017F32121BC37B027D017F3802E2
:0218B5001BC353
:100AA00090E600E054E74410F000000000000090E1
:100AB000E61074A0F000000090E60B7401F090E6E0
:100AC0001274E0F0000000E490E613F000000090E3
:100AD000E61474E2F000000090E61574A0F0000047
:100AE0000090E6D27402F090E6047480F0000000FA
:100AF0007402F00000007406F00000007408F000BA
:100B00000000E4F000000012176990E6187408F085
:100B100000000090E619F000000090E61AF00000D6
:100B20000090E61BF0000000E490E671F075B47FE1
:100B300075A07F90E672F075B6FF75B1FF90E67014
:100B4000F075B2FF75B5FFC28CD2B01222B190E63B
:100B50001074A0F000000090E611F000000090E694
:100B60005EE04408F0000000E490E68DF000000034
:100B700090E65EE04404F0000000E490E7C0F090EE
:100B8000E7C4F0A3F0A3F0A3F090E7F0F090E68FB5
:100B90007440F000000090E65EE04440F000000089
:100BA0007E027F0090F800E4F0A3DFFCDEFA90E61E
:100BB000987402F0000000E490E699F00000007ED6
:100BC000027F0090F800E4F0A3DFFCDEFA90E65E1E
:100BD000E04480F0000000E490E69CF0000000900B
:100BE000E69DF00000007F9AFE12228675270075B0
:100BF00028B47550017551907532107533B875521F
:100C00000675532C1222A990E67AE054FEF0E4FD1A
:100C10007F9012222F7F647E001218B77DFF7F42E3
:100C200012222F7F647E001218B77D827F4E12221F
:100C30002F7540FF43A020E4F54490E782E540F0A3
:100C400090E781E544F01222B1D209754E01753565
:100C500027753610752C0A121B377FD07E071217A6
:100C600052121B377FB87E0B121752121B377FA010
:100C70007E0F121752C201C2B2D2F9C2F8E4F54B8C
:100C800090E7C0E54BF043A01053917F53A0F002D2
:020C9000182525
:0E226300EF2401FBE43EFA7D047F48022130A7
:10205500E544C313FFC374809F9025ABF0E494005F
:102065009025AAF0E544D3940040067540FF43A0AF
:0920750020E544700353A0DF22B2
:10141300E4FC9024FDE0FEA3E02400FDEC3EFC9000
:101423002410E0FEA3E07A002400FFEA3EFEC3EDB1
:101433009FFFEC9EFE9024F2F0A3EFF09024F5E0E2
:101443002FF09024F4E03EF0D3EF9450EE648094B8
:10145300805011C39024F3E094B09024F2E06480B0
:10146300947F50209024F2E0FEA3E0FF7C007D05F2
:10147300120E9B9025AAEEF0A3EFF0E49024F4F073
:10148300A3F080339024F5E025E0FF9024F4E033CB
:10149300FE7C007D0A120EADAA06AB079024F2E093
:1014A300FEA3E0FF7C007D05120E9BEF2BFFEE3ABF
:1014B3009025AAF0A3EFF0D39025ABE094FF9025FD
:1014C300AAE0648094804006E4F0A374FFF0C39024
:1014D30025AAE0648094805004E4F0A3F09025AA48
:1014E300E0FEA3E0FF7C007D02120EADC3747F9F7C
:0714F300F0E49E9025AAF031
:0114FA0022CF
:101CA8007E247FFC1222639024FDE090E7C1F0902F
:101CB80024FEE090E7C2F09025ABE090E7C3F090F7
:101CC80024FBE0600B43A0207540FF12141380032F
:101CD800122055902452E540F07A247B527D017FF2
:101CE8002112214C9024527402F0A37480F07A24BB
:101CF8007B527D027F2812214CE4902452F09025DB
:101D0800ABE0902453F07A247B527D027F28022195
:011D18004C7E
:101314000555E55570020554054DB53610E554B52F
:10132400350B121CA8E4F554F55512211390E7C8A7
:10133400E54EF0A3E52DF0A3E534F0E54D652C7002
:1013440024E54E601414600C14600924FD60050447
:10135400701080001222538009E4FFFE121F7B5399
:10136400A0EFE4F54D200003021412754B0190E741
:10137400C0E54BF0E5A030E7032007F87FAE121973
:10138400F590F00074AAF0A37411F0A374CCF0A348
:1013940074EEF0E490E690F090E6917405F0120F8C
:1013A400B790F00074AAF0A37411F0A374CCF0A366
:1013B40074EEF0E490E690F090E6917405F07FAF5F
:1013C4001219F5C200E4F54B90E7C0E54BF0902408
:1013D400F6E0B40107E53C7003021B37121B377FAC
:1013E400D07E07121752121B377FD07E0712175276
:1013F400121B377FD07E07121752121B377FD07E05
:0F14040007121752121B377FD07E071217522282
:0218FD00D322F4
:0222BA00D3222D
:0222BC00D3222B
:101D820090E680E030E73A00000090E6207402F02E
:101D9200000000E490E621F000000090E6247402C6
:101DA200F0000000E490E625F000000090E62674C2
:101DB20002F0000000E490E627F0000000D202806A
:101DC20016000000E490E620F000000090E6217486
:0F1DD20040F0000000C20290E6BAE0F54CD322C8
:10220B0090E740E54CF0E490E68AF090E68B04F022
:02221B00D322CC
:0822A10090E6BAE0F526D32215
:10221D0090E740E526F0E490E68AF090E68B04F036
:02222D00D322BA
:0222BE00D32229
:0222C000D32227
:0222C200D32225
:10008000E4FFF518F51990E6B9E0244B605224F32B
:10009000700302029924F870030202E124FA70034B
:1000A000020323241D6003020415E490E68AF09005
:1000B000E68BF090E6A0E020E1F990E68BE0E4F535
:1000C000B390E60174CAF0D20000000090E6047418
:1000D00080F00000007402F0000000E4F002041759
:1000E000E490E68AF090E68BF090E6A0E020E1F95B
:1000F00090E68BE0D3943F4024E4F5187440251833
:10010000F582E434E7F583E0FF74122518F582E404
:100110003424F583EFF00518E518B440DF7F8A7EBC
:1001200000122286902412E0FF7E0012228F90247B
:1001300013E075F004A4FFAEF0122298902417E0AB
:10014000C394025013902433E090E6C07005744EBF
:10015000F08016749CF08011902433E090E6C0701B
:1001600005749FF08003749DF0902435E024FF9285
:1001700006902432E024FF9205902436E024FF927A
:1001800008902440E0754200F543A3E0FEA3E07C24
:10019000002400F524EC3EF523902445E09024F65D
:1001A000F0902418E0F53AE53A7003753A0190248E
:1001B0001DE0FEA3E07C002400F528EC3EF527A31B
:1001C000E0FEA3E02400F551EC3EF550902419E048
:1001D000FEA3E02400F533EC3EF532A3E0FEA3E0FD
:1001E0002400F553EC3EF55290244DE0FFE4FDFE73
:1001F000FBFAF97801120EE3A804A905AA06AB07D9
:10020000902423E0FEA3E07C002400FFEC3EFEE40B
:10021000FDEB2FFFEA3EFEED39FDEC38FCC004C0DB
:1002200005C006C00790244EE0FFE4FCFDFEFBFA8B
:100230007901F8120EE3D003D002D001D000EF2BE9
:10024000F54AEE3AF549ED39F548EC38F547902492
:1002500021E0FEA3E07C002400F530EC3EF52F9079
:100260002447E0540FF53CE4FD7F9012222F9024A8
:1002700013E0FCA3E0FDA3E0FEA3E0FF9025011244
:100280000F56902501A3E0FDA3E0FEA3E0FFE4FCF0
:10029000902501120F5602041790E7407429F0A32D
:1002A000741CF0A3740CF0A37426F0A37407F0A3DD
:1002B00074EEF0A37401F0A37403F0A37453F03050
:1002C0000205E4A3F0800690E74974FFF000000007
:1002D000E490E68AF000000090E68B740AF00204D5
:1002E0001790E6BCE0902657F07A267B577D017F79
:1002F0005012214C7A267B577D017F5012214C9061
:10030000E6BEE0FD7AE77B407F50122130E490E6C4
:100310008AF000000090E6BEE090E68BF00000005E
:10032000020417E490E68AF090E68BF090E6A0E0F5
:1003300020E1F990E68BE0F518C29890E740E0C321
:1003400094304014E534242FFFE433FEE0D39FEED5
:100350006480F8748098401190E740E0F4600302F4
:1003600003ECE54E60030203EC43A01090E740E08D
:10037000F4600AE0B4300EE52D64016008D209751E
:100380004E0402041790E740E0C394315003020486
:1003900017E534242FFFE433FEE0D39FEE6480F8AA
:1003A0007480985072E024D1F52E652D6069E0B418
:1003B0000A03752E6190E740E0B40B03752E62903E
:1003C000E740E0B40C03752E6390E740E0B40D0302
:1003D000752E6490E740E0B40E03752E6590E740FB
:1003E000E0B40F03752E66754E02802B90E740E057
:1003F000B4200CE54E700843A010754E058018908F
:10040000E740E0B41104D201800D90E740E0B4125F
:0804100006C2018002D322C3E1
:0104180022C1
:10219B00C0E0C083C082D20C5391EF90E65D740116
:0821AB00F0D082D083D0E032B5
:1021CB00C0E0C083C0825391EF90E65D7404F0D001
:0621DB0082D083D0E03247
:1021E100C0E0C083C0825391EF90E65D7402F0D0ED
:0621F10082D083D0E03231
:101E1800C0E0C083C08285625E85635F855F82851E
:101E28005E83A37402F0855A60855B618561828553
:101E38006083A37407F05391EF90E65D7410F0D0BF
:061E480082D083D0E032DD
:1021B300C0E0C083C082D20E5391EF90E65D7408F5
:0821C300F0D082D083D0E0329D
:1019B800C0E0C083C08290E680E030E720855A5EB0
:1019C800855B5F855F82855E83A37402F0856260B4
:1019D800856361856182856083A37407F05391EF05
:0D19E80090E65D7420F0D082D083D0E03214
:0118FF0032B6
:0122C40032E7
:0122C50032E6
:0122C60032E5
:101EEA00C0E0C083C08290E65EE054FBF0000000D0
:101EFA0090E68F7440F00000005391EF90E65FE0A7
:101F0A004404F090E65EE04404F0D082D083D0E04E
:011F1A003294
:1014FB00C0E0C0F0C083C082C0D075D000C000C0B7
:0D150B0001C002C003C004C005C006C00737
:1015180090E65EE054F7F090E6A1E020E1F990E76C
:1015280080E0FF14601614602624D0603A243460EA
:1015380059146060147062752200805D90E782E043
:10154800F54090E781E0F5449024FBE4F0804A9070
:10155800E782E0902410F090E781E0902411F09069
:1015680024FB7401F0803290E781E07005121B378C
:10157800802790E781E0B40105121F1B801B90E7CC
:1015880081E0B403141220A7800F90E781E024FFC4
:1015980092078005752200D20300000090E68DE4D2
:1015A800F05391EF90E65FE04408F090E65EE04487
:0215B80008F039
:1015BA00D007D006D005D004D003D002D001D00085
:0B15CA00D0D0D082D083D0F0D0E0322F
:0122C70032E4
:0122C80032E3
:0122C90032E2
:0122CA0032E1
:0122CB0032E0
:0122CC0032DF
:0122CD0032DE
:0122CE0032DD
:0122CF0032DC
:0122D00032DB
:0122D10032DA
:0122D20032D9
:0122D30032D8
:0122D40032D7
:0122D50032D6
:0122D60032D5
:0122D70032D4
:0122D80032D3
:0122D90032D2
:0122DA0032D1
:0122DB0032D0
:0122DC0032CF
:0122DD0032CE
:0122DE0032CD
:0122DF0032CC
:0122E00032CB
:0122E10032CA
:0122E20032C9
:0122E30032C8
:0122E40032C7
:0615D5008F1A8C1B8D1C17
:1015DB00531A0753B0F77F0A7E00121752E4F51D1A
:1015EB00F51EC37402951EFFE51AA807088002C3F7
:1015FB0013D8FC30E00543800280035380FD7F0A43
:10160B007E001217524380017F0A7E00121752533D
:10161B0080FE7F0A7E00121752051EE51E70020522
:10162B001DC39403E51D6480948040B6E4F51DF55D
:10163B001EC37409951EFFE51CAE1BA80708800589
:10164B00CEC313CE13D8F930E00543800280035389
:10165B0080FD7F0A7E001217524380017F0A7E00B5
:10166B001217525380FE7F0A7E00121752051EE599
:10167B001E7002051DC3940AE51D6480948040B161
:10168B0043B0087F0A7E0012175253B0F77F0A7ED1
:04169B0000021752E0
:09228600AD07AC06E4FF0215D51A
:09228F00AD07AC067F040215D571
:09229800AD07AC067F010215D56B
:10222F00902452EDF0EFC313FF7A247B527D01020D
:02223F00214C30
:10169F0053A0F043A00C7FEE7E0212175253A0F01E
:1016AF0043A0047FEE7E0212175253A0F043A00610
:1016BF007FEE7E0212175253A0F043A0027FEE7E00
:1016CF000212175253A0F043A0037FEE7E021217AF
:1016DF005253A0F043A0017FEE7E0212175253A087
:1016EF00F043A0097FEE7E0212175253A0F043A0E1
:1016FF00087FEE7E0212175253A0F043A00C7FEE2C
:10170F007E0212175253A0F043A0047FEE7E021206
:10171F00175253A0F043A0067FEE7E0212175253CA
:10172F00A0F043A0027FEE7E0212175253A0F043A7
:10173F00A0037FEE7E0212175253A0F043A0017F49
:03174F00EE7E0229
:10175200EF7803C333CE33CED8F9FFEF4E6007EFF5
:071762001F70F81E80F52244
:0522B100D283D284225B
:10211300C2837F147E00121752C284D2837F147E3F
:0D21230000121752D2847F147E0002175262
:10224100E4FDFC1221130DBD00010CBC0CF5BD0D0C
:01225100F29A
:012252002269
:10110300902501E0FCA3E0FDA3E0FEA3E0FF902413
:10111300F7120F56300502C2B09024F6E0700612A3
:101123001F1B43A0403006030211F1752201E47F27
:10113300E87E03FDFC9024F7E0F8A3E0F9A3E0FACE
:10114300A3E0FBC3120F3250030211DFE522640157
:1011530060030211DF7FDD7E031218B7121CA89013
:1011630024F7E0FCA3E0FDA3E0FEA3E02418FFEED8
:1011730034FCFEED34FFFDEC34FFFC9024F7120F3A
:10118300569024F7E0FCA3A3A3E4FFFEFDEC78183C
:10119300120F4390E7C4EFF09024F7A3E0FDA3A35D
:1011A300E4FFFEE4FC7810120F4390E7C5EFF090E4
:1011B30024F7A3A3E0FEA3E4FFE4FDFC7808120FE9
:1011C3004390E7C6EFF09024F7E0FCA3E0FDA3E033
:1011D300FEA3E0FF90E7C7EFF0021131E522B4016F
:1011E300169024F9E0FEA3E0FF1218B780097522D8
:1011F30001E522640160FA9024F6E0700653A0BF73
:091203001220A7300502D2B0222E
:101C35008F1F8E1E8D1D8C1CE4FFFEFDFCAB1FAAA5
:101C45001EA91DA81CD3120F324057000000E4FF47
:101C5500FEFDE51CFC7818120F4390E6CEEFF00070
:101C65000000E4FFFEE51DFDE4FC7810120F439033
:101C7500E6CFEFF0000000E4FFE51EFEE4FDFC7892
:101C850008120F4390E6D0EFF0000000E51FFF902B
:101C9500E6D1EFF000000075BB04000000E5BB30A5
:031CA500E7FB2238
:081DE1008C1C8D1DAB07AA0646
:101DE900E4FDFCC3ED951DEC951C5022EA90E6D06C
:101DF900F0000000EB90E6D1F000000075BB050093
:0E1E09000000E5BB30E7FB0DBD00010C80D5ED
:011E170022A8
:10207E00AD07AC06000000ED25E0EC3390E6D0F0A5
:10208E00000000ED25E090E6D1F000000075BB04E5
:09209E00000000E5BB30E7FB2265
:1021F700200102C2B230010BD2B27FE87E03121770
:0422070052C2B222EB
:100FB700C20353A0F043A00912174153A0F043A066
:100FC7000312174E53A0F043A0027FF47E011217BD
:100FD7005253A0F043A0067FF47E0112175253A08C
:100FE700F043A0047FF47E0112175253A0F043A0F0
:100FF7000C7FF47E0112175253A0F043A0087FF430
:101007007E011217529024F6E064017024E53C70CB
:101017002053A0F043A0047FF47E0112175253A07F
:10102700F043A00C7FF47E0112175253A0F043A0A7
:10103700081221F7122241754B0290E7C0E54BF0E9
:10104700121103754B0390E7C0E54BF03003030221
:101057001102E4F51AF51BC3E51B9528E51A952738
:10106700500D122113051BE51B7002051A80E8D3EA
:10107700E5439400E5429400400BAD43AC42AF33E7
:10108700AE32121DE1D3E5249400E5239400400716
:10109700AF24AE2312207EE4F518F519C3E51995A0
:1010A70053E5189552502C122000E4F51AF51BC38E
:1010B700E51B953A7480F8651A98500D12211305AF
:1010C7001BE51B7002051A80E60519E51970020574
:1010D7001880C9E4F51AF51BC3E51B9551E51A9568
:1010E70050500D122113051BE51B7002051A80E8ED
:0B10F700AF4AAE49AD48AC47121C35B3
:0111020022CA
:10200000000000E53325E0E5323390E6D0F0000033
:1020100000E53325E090E6D1F000000075BB040038
:0B2020000000E5BB20E7033003F822BE
:101B370053A0F043A00912174153A0F043A003128A
:101B4700174E53A0F043A00212174E53A0F043A024
:101B57000612174E53A0F043A00412174E53A0F0DD
:101B670043A00C12174E53A0F043A00812174E5370
:101B7700A0F043A00912174153A0F043A003121786
:101B87004E53A0F043A00212174E53A0F043A006F5
:101B970012174E53A0F043A00412174E53A0F04360
:101BA700A00C12174E53A0F043A00812174EE4F5ED
:081BB7002590E7CBE525F022A3
:1020A70012172153A0F043A00912174E53A0F04373
:1020B700A00812174E12169F53A0F043A0097525CA
:0820C7000390E7CBE525F022B0
:101F1B0012169F53A0F043A00912174E53A0F04383
:101F2B00A00812174E53A0F043A00C12174E53A04B
:101F3B00F043A00412174E75250190E7CBE525F071
:011F4B002273
:101D19000531E531B40803E4F531E53170057F0893
:101D2900FE804BE531B401067F0A7E008040E53133
:101D3900B402067F027E008035E531B403067F03D5
:101D49007E00802AE531B404067F017E00801FE50C
:101D590031B405067F057E008014E531B406067F9F
:101D6900047E008009E531B4070E7F0C7E00121F46
:091D79007B7F467E001217522206
:10225300E54E600B053EE53E7002053D121D192259
:0822A900E4F56DD2E9D2AF2289
:101E4E0090E678E020E6F9C2E990E678E04480F08A
:101E5E00EF25E090E679F090E678E030E0F990E654
:101E6E0078E04440F090E678E020E6F990E678E0FD
:061E7E0030E1D6D2E9229A
:101EB800A90790E678E020E6F9E56D702390E678CA
:101EC800E04480F0E925E090E679F08D68AF03A959
:101ED800077569018A6A896BE4F56C756D01D3220F
:021EE800C32213
:101E8400A90790E678E020E6F9E56D702590E678FC
:101E9400E04480F0E925E0440190E679F08D68AFF4
:101EA40003A9077569018A6A896BE4F56C756D038A
:041EB400D322C32250
:03004B0002120C92
:10120C00C0E0C083C082C085C084C086758600C023
:10121C00D075D000C000C001C002C003C006C0071A
:10122C0090E678E030E206756D060212F690E678EC
:10123C00E020E10CE56D64026006756D070212F6A4
:10124C00E56D24FE605F14603624FE70030212E725
:10125C0024FC70030212F3240860030212F6AB693B
:10126C00AA6AA96BAF6C056C8F82758300120E4C49
:10127C0090E679F0E56C65687070756D05806B9023
:10128C00E679E0AB69AA6AA96BAE6C8E82758300B5
:10129C00120E79756D02E5686401704E90E678E087
:1012AC004420F08045E56824FEB56C0790E678E0B4
:1012BC004420F0E56814B56C0A90E678E04440F000
:1012CC00756D0090E679E0AB69AA6AA96BAE6C8E7D
:1012DC0082758300120E79056C800F90E678E044DD
:1012EC0040F0756D008003756D005391DFD007D011
:1012FC0006D003D002D001D000D0D0D086D084D07C
:08130C0085D082D083D0E032CD
:10213000121E84E56D24FA600E146006240770F305
:0C214000D322E4F56DD322E4F56DD32228
:10214C00121EB8E56D24FA600E146006240770F3B5
:0C215C00D322E4F56DD322E4F56DD3220C
:03000000021AAB36
:0C1AAB00787FE4F6D8FD75816D021AF218
:100E4C00BB010CE58229F582E5833AF583E022505B
:100E5C0006E92582F8E622BBFE06E92582F8E222A5
:0D0E6C00E58229F582E5833AF583E49322BF
:100E7900F8BB010DE58229F582E5833AF583E8F0AF
:100E8900225006E92582C8F622BBFE05E92582C85B
:020E9900F22243
:100E9B00EF8DF0A4A8F0CF8CF0A428CE8DF0A42E6B
:020EAB00FE2225
:100EAD00C2D5EC30E709B2D5E4C39DFDE49CFCEE60
:100EBD0030E715B2D5E4C39FFFE49EFE120F62C367
:100ECD00E49DFDE49CFC8003120F6230D507C3E462
:060EDD009FFFE49EFE22CF
:100EE300E88FF0A4CC8BF0A42CFCE98EF0A42CFCAE
:100EF3008AF0EDA42CFCEA8EF0A4CDA8F08BF0A42C
:100F03002DCC3825F0FDE98FF0A42CCD35F0FCEB8A
:100F13008EF0A4FEA9F0EB8FF0A4CFC5F02ECD394F
:0F0F2300FEE43CFCEAA42DCE35F0FDE43CFC22BC
:100F3200EB9FF5F0EA9E42F0E99D42F0E89C45F015
:010F4200228C
:100F4300E8600FECC313FCED13FDEE13FEEF13FF8C
:030F5300D8F122B0
:0C0F5600ECF0A3EDF0A3EEF0A3EFF0220E
:101AB700020C92E493A3F8E493A34003F68001F2A7
:101AC70008DFF48029E493A3F85407240CC8C33330
:101AD700C4540F4420C8834004F456800146F6DFFF
:101AE700E4800B0102040810204080900419E47E72
:101AF700019360BCA3FF543F30E509541FFEE493F4
:101B0700A360010ECF54C025E060A840B8E493A3BA
:101B1700FAE493A3F8E493A3C8C582C8CAC583CAE5
:101B2700F0A3C8C582C8CAC583CADFE9DEE780BE9D
:010675000084
:100F6200BC000BBE0029EF8DF084FFADF022E4CC73
:100F7200F875F008EF2FFFEE33FEEC33FCEE9DEC3C
:100F8200984005FCEE9DFE0FD5F0E9E4CEFD22ED82
:100F9200F8F5F0EE8420D21CFEADF075F008EF2FCC
:100FA200FFED33FD4007985006D5F0F222C398FDBD
:050FB2000FD5F0EA225A
:00000001FF
